
D:\STM32\Program\1.11_Odchudzanie\um0427\FWLib\project\RIDE\STM3210E-EVAL\stm32f10x_systick.o:     file format elf32-littlearm
D:\STM32\Program\1.11_Odchudzanie\um0427\FWLib\project\RIDE\STM3210E-EVAL\stm32f10x_systick.o

Disassembly of section .text.SysTick_CLKSourceConfig:

00000000 <SysTick_CLKSourceConfig>:
SysTick_CLKSourceConfig():
D:\STM32\Program\1.11_Odchudzanie\um0427\FWLib\library\src/stm32f10x_systick.c:48
   0:	2804      	cmp	r0, #4
   2:	d104      	bne.n	e <SysTick_CLKSourceConfig+0xe>
D:\STM32\Program\1.11_Odchudzanie\um0427\FWLib\library\src/stm32f10x_systick.c:50
   4:	4a05      	ldr	r2, [pc, #20]	(1c <SysTick_CLKSourceConfig+0x1c>)
   6:	6813      	ldr	r3, [r2, #0]
   8:	f043 0304 	orr.w	r3, r3, #4	; 0x4
   c:	e003      	b.n	16 <SysTick_CLKSourceConfig+0x16>
D:\STM32\Program\1.11_Odchudzanie\um0427\FWLib\library\src/stm32f10x_systick.c:54
   e:	4a03      	ldr	r2, [pc, #12]	(1c <SysTick_CLKSourceConfig+0x1c>)
  10:	6813      	ldr	r3, [r2, #0]
  12:	f023 0304 	bic.w	r3, r3, #4	; 0x4
  16:	6013      	str	r3, [r2, #0]
D:\STM32\Program\1.11_Odchudzanie\um0427\FWLib\library\src/stm32f10x_systick.c:56
  18:	4770      	bx	lr
  1a:	46c0      	nop			(mov r8, r8)
  1c:	e000e010 	.word	0xe000e010
Disassembly of section .text.SysTick_SetReload:

00000000 <SysTick_SetReload>:
SysTick_SetReload():
D:\STM32\Program\1.11_Odchudzanie\um0427\FWLib\library\src/stm32f10x_systick.c:71
   0:	4b01      	ldr	r3, [pc, #4]	(8 <SysTick_SetReload+0x8>)
   2:	6058      	str	r0, [r3, #4]
D:\STM32\Program\1.11_Odchudzanie\um0427\FWLib\library\src/stm32f10x_systick.c:72
   4:	4770      	bx	lr
   6:	46c0      	nop			(mov r8, r8)
   8:	e000e010 	.word	0xe000e010
Disassembly of section .text.SysTick_CounterCmd:

00000000 <SysTick_CounterCmd>:
SysTick_CounterCmd():
D:\STM32\Program\1.11_Odchudzanie\um0427\FWLib\library\src/stm32f10x_systick.c:90
   0:	2801      	cmp	r0, #1
   2:	d104      	bne.n	e <SysTick_CounterCmd+0xe>
D:\STM32\Program\1.11_Odchudzanie\um0427\FWLib\library\src/stm32f10x_systick.c:92
   4:	4a08      	ldr	r2, [pc, #32]	(28 <SysTick_CounterCmd+0x28>)
   6:	6813      	ldr	r3, [r2, #0]
   8:	f043 0301 	orr.w	r3, r3, #1	; 0x1
   c:	e006      	b.n	1c <SysTick_CounterCmd+0x1c>
D:\STM32\Program\1.11_Odchudzanie\um0427\FWLib\library\src/stm32f10x_systick.c:94
   e:	f110 0f02 	cmn.w	r0, #2	; 0x2
  12:	d105      	bne.n	20 <SysTick_CounterCmd+0x20>
D:\STM32\Program\1.11_Odchudzanie\um0427\FWLib\library\src/stm32f10x_systick.c:96
  14:	4a04      	ldr	r2, [pc, #16]	(28 <SysTick_CounterCmd+0x28>)
  16:	6813      	ldr	r3, [r2, #0]
  18:	f023 0301 	bic.w	r3, r3, #1	; 0x1
  1c:	6013      	str	r3, [r2, #0]
  1e:	e002      	b.n	26 <SysTick_CounterCmd+0x26>
D:\STM32\Program\1.11_Odchudzanie\um0427\FWLib\library\src/stm32f10x_systick.c:100
  20:	4b01      	ldr	r3, [pc, #4]	(28 <SysTick_CounterCmd+0x28>)
  22:	2200      	movs	r2, #0
  24:	609a      	str	r2, [r3, #8]
D:\STM32\Program\1.11_Odchudzanie\um0427\FWLib\library\src/stm32f10x_systick.c:102
  26:	4770      	bx	lr
  28:	e000e010 	.word	0xe000e010
Disassembly of section .text.SysTick_ITConfig:

00000000 <SysTick_ITConfig>:
SysTick_ITConfig():
D:\STM32\Program\1.11_Odchudzanie\um0427\FWLib\library\src/stm32f10x_systick.c:117
   0:	b120      	cbz	r0, c <SysTick_ITConfig+0xc>
D:\STM32\Program\1.11_Odchudzanie\um0427\FWLib\library\src/stm32f10x_systick.c:119
   2:	4a05      	ldr	r2, [pc, #20]	(18 <SysTick_ITConfig+0x18>)
   4:	6813      	ldr	r3, [r2, #0]
   6:	f043 0302 	orr.w	r3, r3, #2	; 0x2
   a:	e003      	b.n	14 <SysTick_ITConfig+0x14>
D:\STM32\Program\1.11_Odchudzanie\um0427\FWLib\library\src/stm32f10x_systick.c:123
   c:	4a02      	ldr	r2, [pc, #8]	(18 <SysTick_ITConfig+0x18>)
   e:	6813      	ldr	r3, [r2, #0]
  10:	f023 0302 	bic.w	r3, r3, #2	; 0x2
  14:	6013      	str	r3, [r2, #0]
D:\STM32\Program\1.11_Odchudzanie\um0427\FWLib\library\src/stm32f10x_systick.c:125
  16:	4770      	bx	lr
  18:	e000e010 	.word	0xe000e010
Disassembly of section .text.SysTick_GetCounter:

00000000 <SysTick_GetCounter>:
SysTick_GetCounter():
D:\STM32\Program\1.11_Odchudzanie\um0427\FWLib\library\src/stm32f10x_systick.c:136
   0:	4b01      	ldr	r3, [pc, #4]	(8 <SysTick_GetCounter+0x8>)
   2:	6898      	ldr	r0, [r3, #8]
D:\STM32\Program\1.11_Odchudzanie\um0427\FWLib\library\src/stm32f10x_systick.c:137
   4:	4770      	bx	lr
   6:	46c0      	nop			(mov r8, r8)
   8:	e000e010 	.word	0xe000e010
Disassembly of section .text.SysTick_GetFlagStatus:

00000000 <SysTick_GetFlagStatus>:
SysTick_GetFlagStatus():
D:\STM32\Program\1.11_Odchudzanie\um0427\FWLib\library\src/stm32f10x_systick.c:161
   0:	08c3      	lsrs	r3, r0, #3
   2:	2b02      	cmp	r3, #2
D:\STM32\Program\1.11_Odchudzanie\um0427\FWLib\library\src/stm32f10x_systick.c:163
   4:	bf0c      	ite	eq
   6:	4b05      	ldreq	r3, [pc, #20]	(1c <SysTick_GetFlagStatus+0x1c>)
D:\STM32\Program\1.11_Odchudzanie\um0427\FWLib\library\src/stm32f10x_systick.c:167
   8:	4b04      	ldrne	r3, [pc, #16]	(1c <SysTick_GetFlagStatus+0x1c>)
D:\STM32\Program\1.11_Odchudzanie\um0427\FWLib\library\src/stm32f10x_systick.c:151
   a:	4602      	mov	r2, r0
D:\STM32\Program\1.11_Odchudzanie\um0427\FWLib\library\src/stm32f10x_systick.c:163
   c:	bf0c      	ite	eq
   e:	6818      	ldreq	r0, [r3, #0]
D:\STM32\Program\1.11_Odchudzanie\um0427\FWLib\library\src/stm32f10x_systick.c:167
  10:	68d8      	ldrne	r0, [r3, #12]
  12:	40d0      	lsrs	r0, r2
D:\STM32\Program\1.11_Odchudzanie\um0427\FWLib\library\src/stm32f10x_systick.c:179
  14:	f000 0001 	and.w	r0, r0, #1	; 0x1
  18:	4770      	bx	lr
  1a:	46c0      	nop			(mov r8, r8)
  1c:	e000e010 	.word	0xe000e010
